S020000062696E2F64656D6F70726F675F656B5F6C6D3373383936322E7372656359
S11340005C0400206943000045450000454500006C
S11340104545000045450000454500004545000074
S11340204545000045450000454500004545000064
S11340304545000045450000454500003545000064
S11340404545000045450000454500004545000044
S11340504545000045450000454500004545000034
S11340604545000045450000454500004545000024
S11340704545000045450000454500004545000014
S11340804545000045450000454500004545000004
S113409045450000454500004545000045450000F4
S11340A045450000454500004545000045450000E4
S11340B045450000454500004545000045450000D4
S11340C045450000454500004545000045450000C4
S11340D045450000454500004545000045450000B4
S11340E045450000454500004545000045450000A4
S11340F0EE11AA55F0B587B00120C1F2000045F2D7
S1134100F134C0F20004A0470120C2F20000A0472D
S11341104FF04020032145F20113C0F200039847F9
S113412045F21163C0F20003984701464FF4404042
S1134130C4F200004FF46142602345F6C915C0F291
S11341400005A8470820C2F20000A0474FF4E04051
S1134150C4F20000032145F26903C0F2000398474A
S11341604FF48070C0F21000A0470020C4F2040095
S113417044F25563C0F200039847042303931026C6
S1134180019640F2A460082735463B46741CE218A9
S1134190B0FBF2F14139C9B20A2918D8B5FBF2F1E2
S11341A002FB01F1102912D102930196032B98BF4F
S11341B003931023B3FBF2F204920020C4F2040030
S11341C001A944F27973C0F20003984704E0013B6B
S11341D0DDD16438013ED8D10024C4F20404204661
S11341E044F23573C0F20003984740F267630193C9
S11341F003F5CC730293082303930493204601210F
S113420001AA022344F65D14C0F20004A04707B0DB
S1134210F0BD00BF10B588B040F24403C2F2000301
S11342201B7853BB4FF44040C4F2000045F60D33F5
S1134230C0F200039847B0F1FF3F5FD040F20003A3
S1134240C2F20003187010F0FF0F57D044F2295344
S1134250C0F20003984740F24803C2F2000318601A
S113426040F24403C2F2000301221A7040F24503F3
S1134270C2F2000300221A7040E040F24503C2F289
S113428000031B785C1C4FF44040C4F2000045F668
S11342900D33C0F200039847B0F1FF3F54D040F211
S11342A00003C2F20003185540F24502C2F20002B4
S11342B011780131C9B211701B788B421ED140F2C2
S11342C04403C2F2000300221A7040F20003C2F257
S11342D000035B78FF2B11D140F20003C2F200030C
S11342E09B785BB945F23943C0F20003984705E077
S11342F040F24403C2F2000300221A700020C4F208
S11343000400022144F6AD03C0F20003984710F004
S1134310010F27D001AB07930020C4F20400012150
S113432003AA0B4644F6F534C0F20004A0479DF8F6
S11343300430FF2B16D19DF805309BB945F2394363
S1134340C0F2000398470DE044F22953C0F2000381
S1134350984740F24803C2F200031B686433984252
S1134360C6D8CBE708B010BD10B517498D4640F24A
S11343700002C2F2000240F20003C2F200039A42B9
S113438010D2131D0F4CE41A24F003040434002348
S1134390104645F63C41C0F200015A581A50043305
S11343A0A342FAD109480A494FF000028842B8BF33
S11343B040F8042BFADB44F28D43C0F20003984723
S11343C010BD00BF030000205C040020000000209A
S11343D05C00002010B52020C2F2000045F2F13349
S11343E0C0F2000398474FF4A044C4F202042046EC
S11343F0012145F2B503C0F200039847204601218C
S1134400002245F23903C0F20003984710BD00BFF3
S113441010B544F22953C0F200039847044640F211
S11344204C03C2F200031B68C31AB3F5FA7F2BD303
S113443040F25003C2F200031B7883B940F25003E8
S1134440C2F2000301221A704FF4A040C4F2020029
S1134450114645F23903C0F2000398470FE040F2D9
S11344605003C2F2000300221A704FF4A040C4F2B9
S11344700200012145F23903C0F20003984740F2DB
S11344804C03C2F200031C6010BD00BF08B54FF41A
S11344906070C0F2C01045F25543C0F20003984763
S11344A044F2D533C0F20003984744F2E143C0F22A
S11344B00003984744F2F503C0F20003984744F21E
S11344C01145C0F2000544F21524C0F20004A847C7
S11344D0A047FCE740F25403C2F200031960FEE770
S11344E008B545F21163C0F20003984744F6D3536C
S11344F0C1F26203A3FB0020800945F6F503C0F274
S11345000003984745F6CD03C0F20003984745F6EB
S1134510E103C0F20003984740F25803C2F20003DB
S113452000221A6008BD00BF40F25803C2F2000323
S11345301868704740F25803C2F200031A68013247
S11345401A607047FEE700BF20F480520023C4F2D3
S113455004039A4208D04FF40053C4F2040398426F
S113456014BF002001207047012070474FF480538E
S1134570C4F20403984210D04FF40053C4F204036D
S1134580984208D00023C4F2040398420CBF372099
S11345904FF0FF307047392070473820704700BF14
S11345A082B0016000230193019B042B05DC019B75
S11345B001330193019B042BF9DD02B0704700BF66
S11345C070B582B0044620F47F6020F00F0044F2FE
S11345D06D53C0F2000398470546B0F1FF3F10D178
S11345E045F64430C0F20000F92144F2D543C0F24C
S11345F0000398474EF20413CEF200031B68002612
S113460011E04EF20413CEF200031B68A0F1300255
S1134610012101FA02F212EA030604D045F2F5136D
S1134620C0F20003984723680023019301990429E9
S113463005DC019B01330193019B042BF9DD246804
S11346402EB1284645F24D13C0F200039847204688
S113465002B070BD2DE9F843804644F24953C0F2DC
S11346600003984750B945F64430C0F2000040F2C8
S1134670D91144F2D543C0F20003984740460121C2
S113468044F2A153C0F20003984708F1200544F214
S1134690C156C0F200062C462846B04710F4004F1D
S11346A0F9D108F124094846B02144F2A155C0F2D9
S11346B00005A84708F134000021A84708F1380094
S11346C00021A847012644F2C155C0F2000544F276
S11346D0A157C0F200072046A84710F4004FFAD1B2
S11346E020463146B8470136212EF4D148460C21E4
S11346F044F2A153C0F200039847012644F2C15585
S1134700C0F2000544F2A157C0F200072046A847B2
S113471010F4004FFAD120463146B8470136212E15
S1134720F4D108F1040044F2C153C0F200039847E5
S1134730BDE8F88310B5044644F24953C0F20003BF
S1134740984750B945F64430C0F2000040F23A218F
S113475044F2D543C0F200039847204644F2C153C3
S1134760C0F20003984720F00101204644F2A1530F
S1134770C0F20003984710BDF8B505460C4644F254
S11347804953C0F20003984750B945F64430C0F28B
S113479000004FF4597144F2D543C0F20003984726
S11347A054B945F64430C0F2000040F2653144F299
S11347B0D543C0F2000398472368023B0E2B0AD965
S11347C045F64430C0F2000040F26B3144F2D54368
S11347D0C0F2000398476368013B072B0AD945F6EA
S11347E04430C0F200004FF45C7144F2D543C0F28F
S11347F000039847A368013B032B0AD945F64430CC
S1134800C0F2000040F2753144F2D543C0F2000317
S11348109847E368013BB3F5806F0AD345F644300B
S1134820C0F2000040F27B3144F2D543C0F20003F1
S11348309847284644F2C153C0F2000398470746FC
S1134840284647F0410144F2A156C0F20006B047A1
S11348506368591E090301F4E0412368013B1B020C
S113486003F470631943E368013B03F03F03194306
S1134870A368013B9B01DBB205F10C001943B0476F
S1134880E168013905F11800C1F38311B04717F04D
S1134890010F0CBF27F0400127F04101284644F2E4
S11348A0A153C0F200039847F8BD00BF70B5054698
S11348B00C4644F24953C0F20003984750B945F6F8
S11348C04430C0F2000040F2925144F2D543C0F2A9
S11348D000039847032C3ED8DFE804F00213212F8D
S11348E00435284644F2C153C0F2000398470446F5
S11348F028466FF01F0144F2A153C0F20003984709
S11349002AE005F5807044F2C156C0F20006B047B3
S1134910044605F58270B04744EA00441CE005F5FE
S1134920907044F2C156C0F20006B047044605F543
S11349309270B04744EA00440EE005F5B07044F2CA
S1134940C156C0F20006B047044605F5B270B04740
S113495044EA004400E00024204670BD2DE9F04FF5
S113496089B0054602911646984644F24953C0F26E
S11349700003984750B945F64430C0F2000040F2B5
S11349805F6144F2D543C0F200039847DDF8089014
S113499009F1FF331F2B0AD945F64430C0F2000059
S11349A04FF4CC6144F2D543C0F200039847B8F108
S11349B0040F0AD945F64430C0F2000040F26661A3
S11349C044F2D543C0F20003984705F1200744F2AE
S11349D0C159C0F200094C46B9463846A04710F404
S11349E0004FF9D13C463268B2F5006F3ABFB36864
S11349F0C3F3800C4FF0010CB8F1040F00F2F68001
S1134A00DFE808F003371119290001214FF48077FA
S1134A104FF4005E4FF00009CDF80490CDF80C90EF
S1134A204FF093082DE000210F468E46019103912B
S1134A304FF0930825E000214FF480574FF4005EB7
S1134A4041F6FF79CDF8049009F56049CDF80C9052
S1134A504FF0D30815E001214FF490574FF4005E56
S1134A604FF00009CDF80490CDF80C904FF0930866
S1134A7007E000214FF480778E46019103914FF0B7
S1134A809308B36813F0080F17D0BCF1000F08D0D7
S1134A9070681FFA80F9CDF80C90C0F30C400190B7
S1134AA00BE07068800041F6FC7900EA0909CDF852
S1134AB004904FF00009CDF80C9003F0280028284A
S1134AC002BFDDF8049049F40049CDF8049003F0E6
S1134AD01800182802BFDDF8049049F48049CDF885
S1134AE0049013F0380F1CBF47F480574FF0D308DD
S1134AF048F02008CDF81480BCF1000F0BD01FFA49
S1134B0082F9CDF81890C2F30C4242F4404242EAD2
S1134B100E0207920BE09200C2F30C0242F4004230
S1134B2042EA0E0207924FF00009CDF81890F2689D
S1134B3002F00F0947EA090913F4007F04BF49F0A2
S1134B4080091FFA89F913F0010F18BF49F40069AD
S1134B5013F0020F18BF49F48069F1B1D6F810B010
S1134B6005F13C089246002A17DD0127002644F28D
S1134B70A150C0F20000049040461BF80610BA454C
S1134B802EDD02361BF8073041EA0321049A9047D0
S1134B9008F104080237B245EEDC05F1240005995A
S1134BA044F2A156C0F20006B04705F1280003996B
S1134BB0B04705F12C000199B04705F13000069982
S1134BC0B04705F134000799B04705F1380049466C
S1134BD0B0472046DDF8089009F03F01B04705E0F2
S1134BE044F2A153C0F200039847D6E709B0BDE8E8
S1134BF0F08F00BF2DE9F04F83B006468A46154674
S1134C001C4644F24952C0F20002904750B945F69E
S1134C104430C0F2000040F2C17144F2D543C0F206
S1134C20000398470AF1FF331F2B0AD945F6443095
S1134C30C0F2000040F2C27144F2D543C0F2000356
S1134C40984706F1840B5846002C14BF7B2173212E
S1134C5044F2A157C0F20007B84706F180040AF0F5
S1134C603F0A20465146B84744F2C157C0F20007F4
S1134C702046B84710F4004FFAD106F1880044F2F8
S1134C80C157C0F20007B847019006F18C00B8473D
S1134C90814606F19000B847009006F19400B847A9
S1134CA0804606F19800B8470023AB6083B213F442
S1134CB0807F03D118F4005F03D104E018F4005F8F
S1134CC001D14022AA601FFA88F818F480421FBF5D
S1134CD0C8F30C08009FB9B241EA08411FBF29601C
S1134CE0A96841F00401A96004BFC8F38A012960DE
S1134CF013F4804F1EBFA96841F48071A96013F4B6
S1134D00805F31D09AB1C9F30C02019FB9B241EA74
S1134D1002426A606FF060418A4203D1AA6812F0CD
S1134D20400F13D1AA6842F00802AA600EE0C9F34A
S1134D308A026A6040F2FF718A4203D1AA6812F0C3
S1134D40400F03D1AA6842F00802AA6019F4004F88
S1134D501EBFAA6842F02802AA6019F4804F1EBF41
S1134D60AA6842F01802AA6013F4006F1EBFAA6872
S1134D7042F00102AA6013F4806F1EBFAB6843F0D7
S1134D800203AB6010F4004F04BF0023EB603BD080
S1134D9000F00F00E860AB6813F0400F1CD12F69DE
S1134DA000979C368146B8B14FF00108002744F2C1
S1134DB0C153C0F2000301933046019B9847009B06
S1134DC0D855C14508DD0237000A03F80800043647
S1134DD008F10208B945EFDC5846042144F2A15613
S1134DE0C0F20006B04720465146B04744F2C156CF
S1134DF0C0F200062046B04710F4004FFAD1AB6869
S1134E0043F08003AB60FFE703B0BDE8F08F00BF61
S1134E1020F480534FF40042C4F20502934218BFB9
S1134E20B3F1402F31D04FF4C041C4F200014FF42C
S1134E302042C4F20502934218BF8B4227D04FF49C
S1134E408041C4F202014FF44042C4F2050293428D
S1134E5018BF8B421DD04FF4C041C4F202014FF47D
S1134E606042C4F20502934218BF8B4213D04FF440
S1134E705042C4F203020023C4F20603984218BF4E
S1134E80904214BF00200120704701207047012088
S1134E907047012070470120704700BF70B5044679
S1134EA00E46154644F61163C0F20003984748B90C
S1134EB045F65830C0F20000E42144F2D543C0F274
S1134EC000039847022D09D945F65830C0F2000076
S1134ED0E62144F2D543C0F20003984715F0010FD0
S1134EE004F58063D4F8002414BF3243B2431A603B
S1134EF015F0020F04F58463D4F8202414BF16437C
S1134F0022EA06061E6070BDF8B504460D46174633
S1134F101E4644F61163C0F20003984750B945F6A3
S1134F205830C0F200004FF4DD7144F2D543C0F2B2
S1134F300003984727F008027B1E042A18BF012BA0
S1134F400AD945F65830C0F200004FF4DF7144F23C
S1134F50D543C0F200039847A6F10803052B0BD9EB
S1134F6056B145F65830C0F2000040F2C51144F283
S1134F70D543C0F20003984717F0010F04F5A0636E
S1134F80D4F8002514BF2A43AA431A6017F0020F6D
S1134F9004F20453D4F8042514BF2A43AA431A6024
S1134FA017F0040F04F5A163D4F8082514BF2A43AD
S1134FB0AA431A6017F0080F04F5A363D4F8182560
S1134FC014BF2A43AA431A6016F0010F04F20C53CB
S1134FD0D4F80C2514BF2A43AA431A6016F0020F12
S1134FE004F5A263D4F8102514BF2A43AA431A6017
S1134FF016F0040F04F21453D4F8142514BF2A43F2
S1135000AA431A6016F0080F04F21C53D4F81C25A6
S113501014BF2A43AA431A602EB904F5A563D4F831
S11350202825154305E004F5A563D4F8282522EACC
S113503005051D60F8BD00BF70B504460D46164653
S113504044F61163C0F20003984750B945F658304E
S1135050C0F200004FF4517144F2D543C0F2000392
S1135060984744F8256070BD38B505460C4644F6AB
S11350701163C0F20003984750B945F65830C0F2A6
S113508000004FF4647144F2D543C0F20003984722
S113509028462146022244F69D63C0F20003984745
S11350A0284621460422082344F60974C0F2000469
S11350B0A04738BD38B505460C4644F61163C0F226
S11350C00003984750B945F65830C0F2000040F24A
S11350D0044144F2D543C0F20003984728462146D0
S11350E0012244F69D63C0F20003984728462146F6
S11350F00122082344F60974C0F20004A04738BD15
S113510038B505460C4644F61163C0F200039847CF
S113511050B945F65830C0F2000040F21F5144F235
S1135120D543C0F20003984728462146022244F69C
S11351309D63C0F2000398472846214601220823B4
S113514044F60974C0F20004A04738BD10B5044603
S113515046280AD945F67030C0F200004FF4D571E4
S113516044F2D543C0F200039847042C08D14EF60C
S11351702453CEF200031A6842F480321A6010BD40
S1135180052C08D14EF62453CEF200031A6842F4DB
S113519000321A6010BD062C08D14EF62453CEF20C
S11351A000031A6842F480221A6010BD0F2C08D143
S11351B04EF21003CEF200031A6842F002021A60A3
S11351C010BDA4F110031F2B08D8012202FA03F327
S11351D04FF46142CEF20002136010BD2F2C08D9A7
S11351E0303C012303FA04F44EF20413CEF200031C
S11351F01C6010BD10B5044646280AD945F6703027
S1135200C0F200004FF4F77144F2D543C0F200033A
S11352109847042C08D14EF62453CEF200031A68A2
S113522022F480321A6010BD052C08D14EF62453A6
S1135230CEF200031A6822F400321A6010BD062C64
S113524008D14EF62453CEF200031A6822F48022C9
S11352501A6010BD0F2C08D14EF21003CEF20003D9
S11352601A6822F002021A6010BDA4F110031F2B69
S113527008D8012202FA03F34EF28012CEF20002A1
S1135280136010BD2F2C08D9303C012303FA04F419
S11352904EF28413CEF200031C6010BD30B420F033
S11352A08053A3F58012013A4FF48071C0F21001CB
S11352B08B4218BF012A98BF012040F297804FF417
S11352C00071C0F210014FF48062C0F210029342E8
S11352D018BF8B4208BF012000F088804FF4A04122
S11352E0C2F2100100F16042013A884218BF012A5B
S11352F098BF01207AD90422C2F20002904208BF6A
S1135300012073D01022C2F20002904208BF012093
S11353106CD02022C2F20002904208BF012065D066
S113532020F480148021C2F200014FF48072C2F292
S11353300002944218BF8B4208BF012056D020F0CF
S11353400052B0F1102F18BF402A08BF01204DD0E1
S11353504FF48041C1F200018C4208BF012045D0C6
S1135360B0F1101F08BF012040D04FF48075C1F286
S113537000054FF40071C1F20001884218BFA84231
S113538008BF012032D01025C1F200052021C1F24E
S113539000018A4218BFAA4208BF012026D0082172
S11353A0C1F2100188421CD000F170410139012979
S11353B017D90421C1F200018C4214D0B0F1202F7E
S11353C013D00121C2F2100188420ED04FF4805054
S11353D0C0F21000834218BF082A14BF0020012025
S11353E004E0012002E0012000E0012030BC70470D
S11353F010B5044645F29D23C0F20003984750B906
S113540045F6E830C0F200004FF4FC7144F2D54395
S1135410C0F20003984745F60043C0F20003220F90
S113542053F822301A68A1B2C4F3044401FA04F414
S113543014431C6010BD00BF4EF60C53CEF20003A3
S11354400422C0F2FA521A60FEE700BF01387FF46A
S1135450FDAF704770B504464FF46043C4F20F03C8
S11354601B6813F0E04F0BD04FF46043C4F20F03FA
S11354701A680023C7F2FF031340B3F1805F02D11F
S1135480002CC0F2C3804EF26002C4F20F02116815
S11354904EF27003C4F20F031E6821F4800545F434
S11354A0006546F400601560186011F0020F02D028
S11354B014F0020F05D011F0010F24D014F0010FE5
S11354C021D164F003031D404EF26003C4F20F03C4
S11354D01D60002804DA06F03003302B04D00BE002
S11354E005F03003302B07D14FF4805045F24D4383
S11354F0C0F20003984706E04FF4002045F24D4304
S1135500C0F20003984725F45F5525F0300543F2B7
S1135510F07323401D434DF68F73C7F6FF7333407A
S113552043F4006242F23003C8F200032340134301
S113553004F008024EF25801C4F20F014020086042
S113554053EAC2060AD54EF27003C4F20F031E607A
S11355504EF26003C4F20F031D6009E04EF26003D3
S1135560C4F20F031D604EF27003C4F20F031E60F9
S1135570102045F24D42C0F20002904725F0F86039
S113558020F003000323C0F2C0732340184326F025
S1135590FC5604F0FC510E4314F0804F1FBF40F43E
S11355A0800026F480050023C4F240031ABF234080
S11355B01D4326F0804514F4006F17D14EF25003BA
S11355C0C4F20F031B6813F0400F0BD147F6FF73AF
S11355D04EF25001C4F20F010A6812F0400F01D1DB
S11355E0013BF9D120F4006025F400654EF260031C
S11355F0C4F20F0318604EF27003C4F20F031D606F
S1135600102045F24D43C0F20003984770BD00BF1F
S113561030B44EF26003C4F20F0319684EF2700303
S1135620C4F20F031A68002AB4BF02F0700301F039
S11356303003202B71D003D87BB1102B16D037E167
S1135640602B00F0C180702B00F0BB80302B08BFB2
S113565003F5EA4300F0CF802AE145F68C33C0F22B
S11356600003C1F3841053F82030C4E04FF46043C6
S1135670C4F20F031B6813F0E04F04BF4EF2C013D3
S1135680C0F2E40300F0B7804FF46043C4F20F03A8
S113569018680023C7F2FF030340B3F1805F00F0F2
S11356A096804FF46043C4F20F0318680023C7F2D6
S11356B0FF0303400020C1F20100834208D14FF4EC
S11356C06043C4F20F031B689BB2022B00F084807A
S11356D04FF46043C4F20F0318680023C7F2FF03BA
S11356E003400020C1F2030083421CBF4FF4105357
S11356F0C0F2F4037FD14FF46043C4F20F031C687B
S1135700A4B24FF4D853C0F2B7034FF41050C0F210
S1135710F400002C18BF03466DE04FF46043C4F25C
S11357200F031B6813F0E04F04BF43F67003C0F28D
S1135730390360D04FF46043C4F20F0318680023A8
S1135740C7F2FF030340B3F1805F4AD04FF46043D4
S1135750C4F20F0318680023C7F2FF0303400020BC
S1135760C1F20100834207D14FF46043C4F20F0336
S11357701B689BB2022B39D04FF46043C4F20F0371
S113578018680023C7F2FF0303400020C1F203009E
S113579083421CBF4FF41063C0F23D032BD14FF47E
S11357A06043C4F20F031C68A4B24CF2C063C0F29D
S11357B02D034FF41060C0F23D00002C18BF0346C7
S11357C019E04FF4004316E04FF4800313E04EF267
S11357D0C013C0F2E4030EE04FF4D853C0F2B70391
S11357E009E043F67003C0F2390304E04CF2C063ED
S11357F0C0F22D03FFE7002A03DA12F4006F03D08E
S113580058E011F4006F5AD14EF26400C4F20F0054
S113581000684FF46044C4F20F04246814F0E04FAD
S11358200BD04FF46044C4F20F0425680024C7F27F
S1135830FF042C40B4F1805F0AD1C0F34814023451
S113584004FB03F300F01F040234B3FBF4F309E098
S1135850C0F3481404FB03F300F01F040134640094
S1135860B3FBF4F310F4804F18BF5B0810F4004F3F
S113587018BF9B08002AA8BF41F4800112DA12F075
S1135880804F09D012F4006F06D15B00C2F3865238
S11358900132B3FBF2F016E0C2F3C5500130B3FBA2
S11358A0F0F010E0C1F3C3500130B3FBF0F00AE0B4
S11358B0002008E011F4800FE1D1184603E011F450
S11358C0800FEFD1184630BC704700BF4EF2100372
S11358D0CEF200031A6842F005021A60704700BF56
S11358E04EF21003CEF200031A6842F002021A606C
S11358F0704700BF10B5441EB4F1807F09D345F64C
S11359000C40C0F20000D02144F2D543C0F20003A1
S113591098474EF21403CEF200031C6010BD00BF82
S113592020F480524FF44043C4F200039A4208D05A
S11359304FF46043C4F20003984214BF00200120D6
S113594070470120704700BF10B5044645F6211387
S1135950C0F20003984750B945F62440C0F2000055
S11359604FF4CF7144F2D543C0F200039847E36A81
S113597043F01003E362236B43F4407343F00103E9
S1135980236310BD10B5044645F62113C0F200038D
S1135990984750B945F62440C0F200004FF4DF7137
S11359A044F2D543C0F200039847A36913F0080FEB
S11359B0FBD1E36A23F01003E362236B23F4407307
S11359C023F00103236310BDF8B504460E461546C3
S11359D01F4645F62112C0F20002904750B945F621
S11359E02440C0F2000040F20D1144F2D543C0F24D
S11359F00003984755B945F62440C0F200004FF41F
S1135A00877144F2D543C0F2000398474FF46042D3
S1135A10C4F20F02136813F0E04F08BF102340D004
S1135A204FF46043C4F20F031A680023C7F2FF0364
S1135A301340B3F1805F08BF102332D04FF46043AA
S1135A40C4F20F031A680023C7F2FF0313400022B5
S1135A50C1F20102934209D14FF46043C4F20F032F
S1135A601B689BB2022B08BF10231AD04FF460436B
S1135A70C4F20F031A680023C7F2FF031340002285
S1135A80C1F20302934218BF08230AD14FF46043C2
S1135A90C4F20F031B689BB2002B0CBF1023082316
S1135AA0FFE705FB03F3B3420AD945F62440C0F2ED
S1135AB0000040F20F1144F2D543C0F200039847AE
S1135AC0204645F68512C0F200029047B6EB051F4A
S1135AD0236B3DBF43F0200323636D0823F02003B1
S1135AE028BF2363F600B6FBF5F50135EB096362C5
S1135AF0C5F34505A562E7620023A361204645F688
S1135B004913C0F200039847F8BD00BF10B504461E
S1135B1045F62113C0F20003984750B945F62440D6
S1135B20C0F2000040F2094144F2D543C0F2000340
S1135B309847A36913F0100F0CBF20684FF0FF3093
S1135B4010BD00BF6C69622F6472697665726C69FE
S1135B50622F63616E2E63006C69622F64726976D2
S1135B6065726C69622F6770696F2E6300000000B4
S1135B706C69622F6472697665726C69622F696EF2
S1135B80746572727570742E6300000040420F00D9
S1135B9000201C0080841E0000802500999E360091
S1135BA00040380000093D0000803E0000004B002A
S1135BB0404B4C0000204E00808D5B0000C05D0017
S1135BC00080700000127A0000007D00809698002A
S1135BD0001BB7000080BB00C0E8CE00647ADA0086
S1135BE00024F4000000FA006C69622F6472697684
S1135BF065726C69622F73797363746C2E63000031
S1135C0000E10F4004E10F4008E10F406C69622F8E
S1135C106472697665726C69622F737973746963EF
S1135C206B2E63006C69622F6472697665726C69AD
S10F5C30622F756172742E630000000086
S9034000BC
